:100000000C94CD040C94F5040C94F5040C94F504B4
:100010000C94F5040C94F5040C94F5040C94F5047C
:100020000C94F5040C94F5040C94F5040C94F71B53
:100030000C94F5040C94F5040C94F5040C94F5045C
:100040000C94AD1B0C94F5040C94F5040C94F5047D
:100050000C94F5040C94F5040C94F5040C94F5043C
:100060000C94F5040C94F50408080008001838B442
:1000700000100808FF81FFA3C5FF81FF08080024C6
:10008000187E3C7E3C0008080000183C1824000044
:10009000450084010000484947482053434F5245DA
:1000A0005300177361766500166261636B00157407
:1000B000797065000A0A0A153A6F6B617920163A61
:1000C0006564697400596F7520656E746572656446
:1000D0000A0045004001418149788D782C050000D7
:1000E00045000181307F000045002C0100004500E3
:1000F00054010000450049707C014D782C0400003B
:100100004F7574206F6620616D6D6F210045004C46
:10011000010000F400EE00E800E000D200450049D4
:10012000784D78280A0000526566696C6C65642019
:1001300021000500400150015C01700180016C014B
:1001400054016001740184014C015C0168017C016F
:100150008C01000055706772616465642021004560
:1001600061726E20243520666972737400153A61DD
:100170006363657074002063726162732E000A62AB
:1001800079206B696C6C696E670A00596F75206D18
:1001900061646520240047414D45204F564552215A
:1001A000004E4557204849474853434F5245004762
:1001B000414D45204F564552210045006405000041
:1001C0000808000C1C181000000008086C928244FB
:1001D0002810000008086CFEFE7C3810000008089B
:1001E000003C5A7E7E7E3C00153A73686F6F742027
:1001F000163A72756E004C4554275320474F210024
:100200000101FF030101F7034D61696E204D656E29
:10021000750053797374656D20496E666F00486987
:1002200067682073636F72657300526573746172DF
:100230007400506C61790004020002000000002488
:100240000027002A0000000000250028002B0005E0
:10025000008930080238024978681400002F0056DF
:100260006F6C756D653A004261636B6C69676874A9
:100270003A004C696768743A002F34004261742078
:100280006C766C3A006D56004261743A0005077F47
:100290004141417F3E5B4F5B3E3E6B4F6B3E183CA6
:1002A000783C18183C7E3C181C577D571C1C5E7F00
:1002B0005E1C007E43437E007E73737E007E7F7FE4
:1002C0007E7F4141417F30483A060E062979290652
:1002D0007F4141417F60703F02042A1C361C2A7F07
:1002E0003E1C080000081C3E7F14227F22143C3C68
:1002F0003C7EFF18423C817E3E6375633E3E616BEF
:10030000633E3E636B6B3E04027F020410207F203D
:100310001008082A1C08081C2A0808143E55412207
:10032000637569756310181C1810040C1C0C04000C
:100330000000000000005F00000007000700147FBD
:10034000147F14042A7F2A10231308646236495646
:1003500020500008070300001C2241000041221C1D
:10036000002A1C3E1C2A08083E080800E060000025
:100370000808080808006060000060100804033ED8
:100380005149453E00427F40006251494946214162
:10039000494D331814127F1027454545393C4A49C9
:1003A0004930412111090736494949360649492949
:1003B0001E00002400000080640000081422410098
:1003C0001414141414004122140802015909063EA1
:1003D000415D594E7C1211127C7F494949363E419C
:1003E0004141227F4141221C7F494949417F0909FE
:1003F00009013E414151327F0808087F00417F4199
:10040000002041413F017F081422417F404040408D
:100410007F020C027F7F0204087F3E4141413E7F04
:10042000090909063E416141BE7F0919294626494D
:1004300049493201017F01013F4040403F1F2040B8
:10044000201F3F4038403F631408146303047804BE
:10045000036151494543007F414100030408106096
:100460000041417F000402010204808080808000FE
:100470000307080020545478407F28444438384407
:10048000444428384444287F3854545418087E097A
:10049000090218A4A49C787F0804047800447D40D5
:1004A00000006080847D7F1010284400417F400060
:1004B0007C047804787C080404783844444438FC8C
:1004C0001824241818242418FC7C08040408085450
:1004D000545420043F4444203C4040207C1C204095
:1004E000201C3C4020403C44281028444C909090D4
:1004F0007C4464544C44000836410000007F0000F6
:100500000041360800180408100C7F4141417F3239
:10051000022A021E02120208021753440016137820
:1005200000161314001510200015201000540A03A3
:10053000E181867F3E186D830F0F0E018386603345
:10054000186DC3198F1803C38E6033186DE330CF55
:100550001803C39E603630CDE360CF3006C79E7E61
:100560003E30CDB360CF300CC6F6603330D9B660C4
:10057000CF33CFCCF66061B0DB1E60CF30D86CE6F5
:10058000C061B0DB1E618F19986CC6C063B19B0E51
:10059000330F0FB078C6FF7E1F1B061E0F4024FFCF
:1005A000FFFFFFFFFFFFFF800000000001414180CF
:1005B0000001800604141180000180060080818003
:1005C000000180060000418F3F79B9EF9E7E1199AE
:1005D000BBCDFB3633762199B30D983633664598FB
:1005E000307D99F63360039830CD9B363361419866
:1005F00030CD9B3633641599B0DD9B76336089CF5F
:1006000030FDF3F39E60418000000000000515A05E
:10061000000000002080A1C000180C00000FF59021
:1006200000245280F00813D002AC5681F80FF199E3
:100630004334DAE1F80A359542255281F80C59DD48
:10064000C219CC61680FF18040000000F0081580ED
:1006500080000000000FF1C00000000600000580CF
:100660000000000F000003C0000000060000019021
:10067000000000090000058000000000000009C122
:100680004000000000000193D0000000000005A31E
:10069000E000000006000183E00545400F054583AA
:1006A000D00202000602038140014140090141805D
:1006B00000041410000415FFFFFFFFFFFFFFFF0001
:1006C000F6E8DBCFC3B8AEA49B928A827B746E68D7
:1006D000625C57524E4945413E3A3734312E2C29FF
:1006E000272523210A0A153A49676E6F7265006D46
:1006F000560A0A504C45415345205455524E204FFE
:10070000464620004C4F57204241545445525921EF
:10071000200003053F213F1208120A100A0E1C0E8A
:100720000C1E0C141A14161F161E131E1E1B1E1E42
:100730001F1E3F213F3A2F3A173D173F213F181FF9
:1007400002040A041F0E04040E1F0A1F0A0E0E1FC5
:1007500004110E2E252E2F2A2E262929021F0208CB
:100760001F08150E04040E150E15151B151B040687
:1007700004040C040000000017000300031F0A1FFC
:1007800016371A1904130A153A000300000E111146
:100790000E000A040A040E040030000404040010D1
:1007A000001804031F111F121F101D151711151F0C
:1007B00007041F17151D1F151D01011F1F151F17EA
:1007C000151F000A00003200040A110A0A0A110A61
:1007D000040115020E11171E051E1F150A0E110A1F
:1007E0001F110E1F15111F05010E111D1F041F11D2
:1007F0001F1108100F1F041B1F10101F061F1E04BF
:100800000F0E110E1F09060E112E1F051A121509C3
:10081000011F011F101F0F180F1F0C1F1B041B03AC
:100820001C03191513001F11030418111F000201E6
:10083000022020200001020C121E1F120C0C1212AA
:100840000C121F0C1A14041E05242A1E1F021C144D
:100850001D1020201D1F0814111F101E041E1E0233
:100860001C0C120C3E0A040C123E1E040214160A42
:10087000020F120E101E0E100E1E081E120C122653
:10088000281E322A26041E21001F00211E040102F8
:10089000013F213F172B152010204C4F414445525A
:1008A00000172B16201314004D47343200525047C6
:1008B00000414B343700503930002E33353700CFEC
:1008C000CF804001FC39E00C06871FC3C181013C89
:1008D0003307E08409C1CF0808542014418804512B
:1008E0000A696E6600BA08B608B108AD08A808051E
:1008F0000038016801000005006801380100000AA5
:100900004E6F2053442063617264206F720A6E6FD1
:10091000204C4F414445522E4845580A0A153A4545
:10092000786974001D20466C617368696E670A20DF
:10093000206C6F616465722E2E2E0A0A444F4E277A
:1009400054205455524E204F4646210000000000CE
:100950002300260029000404040404040404020201
:10096000020202020303030303030102040810202E
:100970004080010204081020010204081020000039
:10098000000800020100000304070000000000004E
:1009900000004500680100004E2911241FBECFEF62
:1009A000D8E0DEBFCDBF11E0A0E0B1E0E0E6F7E5C2
:1009B00002C005900D92AA35B107D9F725E0AAE546
:1009C000B1E001C01D92AA37B207E1F714E0CDEC07
:1009D000D4E004C02197FE010E949D29CC3CD107A0
:1009E000C9F70E9481240C94AE2B0C940000DF9276
:1009F000EF92FF920F931F93CF93DF930E943314D4
:100A00008823E1F362E070E080E090E00E948219C8
:100A1000675F6093480562E070E080E090E00E94CC
:100A200082196093490566E970E08FE395E00E94C2
:100A30002F1A109246051092480580914405809324
:100A40004905C9E9D2E003EA12E0DD24D3947E012E
:100A500088819981892B31F46DE28FE395E00E94C2
:100A6000A61905C0B8018FE395E00E94D1198091C5
:100A70004305982F990F890F81958C5A80934805CB
:100A800080914405D89E802D11248093490522969B
:100A9000F701808191810E94AF21D394055F1F4FA0
:100AA000F6E0DF12D4CF80910605813059F486E15B
:100AB00095E0DF91CF911F910F91FF90EF90DF9024
:100AC0000C94841C80910705813089F3809108057E
:100AD000813009F093CFEBCF2F923F924F925F92EC
:100AE0007F928F929F92AF92BF92CF92DF92EF92BE
:100AF000FF920F931F93CF93DF9300D000D0CDB719
:100B0000DEB7782E90E08C0109581D4FD8014C912A
:100B1000880F991FFC01E95AFD4F6F0160817181B7
:100B20009C01295C3D4F7901242FD7018D919C9127
:100B30000E945D1F81114DC09091DC02E7E5F2E05B
:100B4000FC83EB8327E332E03A832983E7E7F2E093
:100B5000160127012E2FA7E7B2E02A1B2917C8F597
:100B6000721641F12081AB81BC81CD90DC90A981CE
:100B7000BA816D917C91D8014C9150E0D101ED90FA
:100B8000FC90D201AD90BC904501840E951E681575
:100B9000790584F430E0620F731FA616B70654F48B
:100BA0004E0D5F1DC416D5062CF42C0D3D1DE2160E
:100BB000F30674F031962B813C812E5F3F4F3C83CE
:100BC0002B8349815A814E5F5F4F5A834983C2CF3D
:100BD00081E00F900F900F900F90DF91CF911F91B8
:100BE0000F91FF90EF90DF90CF90BF90AF909F90CC
:100BF0008F907F905F904F903F902F9008959F929D
:100C0000AF92BF92CF92DF92EF92FF920F931F931A
:100C1000CF93DF93982EC82FD0E0DE01A958BD4FA7
:100C200084E08C93FE01E654FE4F8AE0808380913D
:100C3000DA01811112C09091DB01292F30E02330BD
:100C4000310514F0915001C091E09093DB01909335
:100C5000DA0186E08C9384E680838E01000F111FF9
:100C6000A801495C5D4F7A01095A1D4F30E8A32E57
:100C7000B12C40E6C42ED12C60E270E080E090E020
:100C80000E948219660F771F660F771FF701718325
:100C9000608368E170E080E090E00E948219660F56
:100CA000771F660F771FF80171836083892D0E947B
:100CB0006C058111E1CFF7018081918180589F4FB0
:100CC00020918B0230918C02821B930BB5010E9404
:100CD00075298435910584F2F80120813181205AEB
:100CE0003F4F8091890290918A02A901481B590BBC
:100CF000CA01B6010E947529C0970CF4BDCF0E94AD
:100D0000272BC452DE4F24E030E040E050E00E9448
:100D10004B2B688381E0DF91CF911F910F91FF9062
:100D2000EF90DF90CF90BF90AF909F900895CF93BA
:100D3000DF93EC01FB01DA018C91813099F058F0DE
:100D40008230B9F0833001F588819981820F911D3D
:100D500027FD9A9517C080819181821B910927FDFB
:100D600093950DC088819981821B910927FD9395E8
:100D700009C080819181820F911D27FD9A959183F1
:100D8000808302C0998388838881998180589F4F8E
:100D900060E870E00E947529998388838081918141
:100DA000805A9F4F60E670E00E947529918380838E
:100DB000DF91CF910895CF93DF93FB01EA0140913A
:100DC0008B0250918C02841B950B089697FD03C0F3
:100DD0008F77992706C060E870E00E9475298058D7
:100DE0009F4F0897998388838091890290918A0206
:100DF000AF01481B590BCA01089660E670E097FDE9
:100E000003C00E94752904C00E947529805A9F4F13
:100E1000AC0148505109F90151834083888199817F
:100E20008535910524F481E0413351050CF080E0D3
:100E3000DF91CF9108952F923F924F925F926F92E0
:100E40007F928F929F92AF92BF92CF92DF92EF925A
:100E5000FF920F931F93CF93DF9300D000D01F9288
:100E6000CDB7DEB7382EC82ED12C70E0CB01825E14
:100E70009D4F2C01DC018C9190E0F601E654FE4F71
:100E8000DC01A05FBE4F20802C91221A2082FC0141
:100E9000E55FFE4F3081F601E958FD4F5F0180812B
:100EA000863011F436953695CB018C5E9D4F7C01D2
:100EB0008601000F111FD801A95ABD4F3D01F8014D
:100EC000E95CFD4F4F01232FA701BD01CF013D83F9
:100ED0000E949706832D0E946C053D81882339F07E
:100EE000232F2195A701B301C4010E949706F601A3
:100EF000E452FE4FD7018C9190E0029683709927BF
:100F0000808312140CF49FC080917805909179052C
:100F1000019690937905809378058091DA029091FB
:100F2000DB0201969093DB028093DA028091DA0172
:100F300081508093DA01F2018081833039F040E002
:100F400060E970E086E195E00E944B1CD5018C9130
:100F5000863049F4809178059091790504969093B4
:100F6000790580937805F801E95AFD4F2081318198
:100F7000F801E95CFD4F40815181EAECF1E080E04D
:100F800090E0619161111EC0FC01E653FE4F61E0EB
:100F900060837C01EE0CFF1CF701E656FE4F518387
:100FA0004083F701E658FE4F3183208365E070E00F
:100FB00080E090E00E948219F701E65AFE4F7183AB
:100FC000608304C0019680319105D9F6F801E95A91
:100FD000FD4F60817181F801E95CFD4F9E012F5F3B
:100FE0003F4FAE014D5F5F4F808191810E94DB06D4
:100FF000882361F0F50120812F5F498141506B8189
:101000006150022F8FE395E00E94021E832D0E9403
:10101000FF052091DC022031B0F48091DA0290913A
:10102000DB0266E070E00E9475296D5F7F4F822FC2
:1010300090E0681779073CF081E0820F8093DC0232
:10104000822F0E94FF050F900F900F900F900F902E
:10105000DF91CF911F910F91FF90EF90DF90CF9094
:10106000BF90AF909F908F907F906F905F904F90C8
:101070003F902F900895FF920F931F93CF93DF938C
:1010800000D000D0CDB7DEB7F12C8091DC02F8168D
:1010900098F50F2D10E0C801880F991FFC01E95A3F
:1010A000FD4F60817181FC01E95CFD4F9E012F5F66
:1010B0003F4FAE014D5F5F4F808191810E94DB0603
:1010C0008823C1F0F801E958FD4F9081F801E452FE
:1010D000FE4F69818B81963031F06250208146E865
:1010E00050E0825005C0615020814CE750E08150B3
:1010F0000E94DF20F394C9CF0F900F900F900F90B4
:10110000DF91CF911F910F91FF900895CF93DF93BF
:1011100000D000D0CDB7DEB76091350270913602B5
:101120009E012F5F3F4FAE014D5F5F4F80913302B5
:10113000909134020E94DB06882341F022E730E0E0
:1011400049816B818FE395E00E949D1C0F900F9069
:101150000F900F90DF91CF9108950F931F93CF932E
:10116000DF9300D000D0CDB7DEB711E060E170E0D2
:1011700080E090E00E94821983E0660F771F8A95D5
:10118000E1F770933402609333026CE070E080E02A
:1011900090E00E94821993E0660F771F9A95E1F71D
:1011A000709336026093350228E048E08091330264
:1011B000909134020E945D1F082F6091350270915A
:1011C00036029E012F5F3F4FAE014D5F5F4F809112
:1011D0003302909134020E94DB068111C7CF0117C0
:1011E00029F20F900F900F900F90DF91CF911F91E8
:1011F0000F9108952F923F924F925F926F927F923C
:101200008F929F92AF92BF92CF92DF92EF92FF9216
:101210000F931F93CF93DF93CDB7DEB72D970FB604
:10122000F894DEBF0FBECDBF2091780530917905CF
:101230008091A1029091A202821793070CF034C210
:10124000E0E8F7E7859194918130904CD1F06DE81A
:1012500072E08FE395E00E94891C10924505109280
:10126000D902A0E3CA2EB4E5DB2E12E0F12EE12C68
:1012700010E00AEF502E82E0682E712C90E3492E88
:1012800066C0EBE8F7E78491DF01AC5BB4478C9371
:101290003196E53987E7F807B1F7D9CF8091050591
:1012A0008F3F09F059C0809103058F3F09F059C065
:1012B000809104058F3F09F059C0809102058F3F4E
:1012C00009F059C090E1E9125BC0E12CE8E0FE12A0
:1012D0005CC0F12C909144058091430580958E9DD2
:1012E000802D1124895DAD2CDD0CBB08A80EB11C2E
:1012F00087FDBA94B7FE03C0FFEFAF1ABF0AB594DB
:10130000A7943A2CDA2C84E1891B90959F9D800D3F
:1013100011248C2CCC0C9908880E911C87FD9A9472
:1013200097FE03C02FEF821A920A95948794282C77
:10133000C82C80910605813009F044C01A30D4F5DC
:101340002E2D80E1F89E200D1124211123C00E9432
:1013500033148823E1F3A2CF8370813009F0A3CF47
:101360001DC28370813009F0A3CF1CC2837081300D
:1013700009F0A3CF1BC28370813009F0A3CF1AC23A
:10138000E7FEA4CFFFE0EF2EA1CFF7FEA3CFE7E06B
:10139000FE2EA0CF2A30D9F22D30C9F2812F012E96
:1013A000000C990BFC01E153FD4F2083FC01E0533D
:1013B000FD4F10821F5F86E195E00E94841C1C3067
:1013C0000CF01BE080910705813071F4115086E12B
:1013D00095E00E947F1C17FDF1C1E12F012E000C4A
:1013E000FF0BE153FD4F108280910805813051F4CD
:1013F000E7C180910705813009F0E6C186E195E0FB
:101400000E947F1C70E050E030E0232F270F809176
:101410004405452F589F400D1124420D80914305EE
:10142000632F389F600D1124630D01E08FE395E079
:101430003B875C877D870E942B1E3B853F5F5C85D9
:101440007D85303111F75F5F705F5830E9F680912C
:1014500043059A2D859D900D1124892F82508093EC
:101460004805809144058F5F880D809349056EEA99
:1014700070E08FE395E00E94AD1980914305EA2D5D
:10148000859DE00D11248E2F825080934805809118
:101490004405880F8E5F880D8093490568EA70E0E7
:1014A0008FE395E00E94AD1980914305FA2D859D4B
:1014B000F00D11248F2F82508093480580914405B0
:1014C00090E00196982F990F890F880D8093490518
:1014D00062EA70E08FE395E00E94AD1910925F051B
:1014E00010926005809144054F2DF89E400D112407
:1014F0004250480D809143056E2DE89E600D1124E9
:1015000061506A0D27E08FE395E00E94DF1DBB2448
:10151000B394B0925F05B09260053091440540915C
:101520004305E42FF0E025E0230F4E5FCF01019744
:10153000B3010E947529480F6F2DF39E600D112491
:101540006350680D8E2DEE9E800D112482508A0D01
:101550000E945723809144054EE2481B24E560E039
:101560008FE395E00E94DF1D10925F0510926005E9
:101570008091440501E0080F4FE2481B24E560E03C
:101580008FE395E00E94021E109248058091440569
:10159000242D281B20934905B0925F05B092600569
:1015A0006FEC72E08FE395E00E94D11980916205A3
:1015B00090916305A0916405B091650587709927A6
:1015C000AA27BB270497A105B10508F0C0CE1A30A1
:1015D0000CF0BDCE80914405442D481B609143051D
:1015E000169F602D112401E02FE58FE395E00E9406
:1015F0002B1EADCE5801FBE0AF1AB108B501CE01EC
:1016000001960E94D22AB801C5010E94D22ABE01C9
:101610006F5F7F4FC8010E94D22AF70171826082FA
:10162000938282828501F2E0033A1F0749F0F701B5
:10163000929082907F016280738086149704D4F226
:1016400059E9A52E52E0B52E0AE010E0E12CF12C6C
:1016500048018AE0881A9108F601EE0DFF1D6081AD
:10166000C701880D991D0E943D2B2FEFE21AF20A47
:101670008AE0E816F10481F7F5016081C8010E9453
:101680003D2BF5016181F2E0AF0EB11CC80101965E
:101690000E943D2B045F1F4F2BE0C20ED11C06346D
:1016A0001105A1F60E94F7041092790510927805B1
:1016B0001092DB021092DA021092EA028FE097E2B7
:1016C0009093E8028093E7021092E9021092870259
:1016D00086E08093880280E18093DB018093DA01C9
:1016E00084E08093DC024FE0E42E47E2F42E60E1D8
:1016F00070E080E090E00E94821923E0660F771F7F
:101700002A95E1F77093900260938F026CE070E08D
:1017100080E090E00E94821933E0660F771F3A95CF
:10172000E1F770938E0260938D0226E046E080918F
:101730008F02909190020E945D1F8111D8CF8091FD
:101740008F0290919002879790938C0280938B02E6
:1017500080918D0290918E02459790938A0280939A
:1017600089029091DC02A7E3B2E0E7E5F2E080E0D5
:10177000891731F0ED92FD92E192F1928F5FF8CFEF
:1017800010E08091DC02181708F050C0812F0E94F1
:10179000FF05882309F4ABCF1F5FF3CFF3940E94BA
:1017A000E82181CDFA940E94E82182CDE3940E9441
:1017B000E82183CDEA940E94E82184CD10E014CE84
:1017C00086E195E00E94841C0E9433148823E1F393
:1017D00065EC70E08FE395E00E942F1A6FEC72E0E9
:1017E0008FE395E00E94D11964EB70E08FE395E000
:1017F0000E942F1A80910605813009F0FACD86E10A
:1018000095E00E94841C80917805909179059093D1
:10181000A2028093A10281EAE82E82E0F82E0FEC6A
:1018200012E093EAC92E92E0D92E01CF0E94AD08B2
:10183000E8E2F2E08AE08E0F11928E13FDCFEAEC1F
:10184000F1E080E18E0F11928E13FDCF10923202E3
:101850002D960FB6F894DEBF0FBECDBFDF91CF91AE
:101860001F910F91FF90EF90DF90CF90BF90AF90BE
:101870009F908F907F906F905F904F903F902F90B0
:101880000895EF92FF920F931F93CF93DF9300D0B1
:1018900000D0CDB7DEB78AECE82E81E0F82E00E06C
:1018A00010E0F7018081882319F1F801E658FE4F16
:1018B000608171819E012F5F3F4FAE014D5F5F4F91
:1018C000F801E656FE4F808191810E94DB06882355
:1018D00069F0698162508B81F801E65AFE4F2081E0
:1018E00048E650E082500E94DF2002C0F7011082DB
:1018F000FFEFEF1AFF0A0E5F1F4F0032110589F646
:101900000F900F900F900F90DF91CF911F910F913B
:10191000FF90EF900895FC01643508F053C0403308
:1019200008F050C090A1742F759575957595262F68
:10193000062E000C330B542F57709230A1F4F9018E
:10194000EF50FD4F84E57802E00DF11D11248081F8
:1019500090E0052E02C0959587950A94E2F7809550
:10196000982F91700AC0933041F484858170462786
:1019700040954170841303C014C0911112C084E5D6
:101980007802200D311D1124F901EF50FD4F81E047
:1019900090E001C0880F5A95EAF7809590818923DD
:1019A00010C084E57802200D311D1124F901EF509B
:1019B000FD4F81E090E001C0880F5A95EAF79081D1
:1019C000892B808308958F929F92AF92BF92CF927E
:1019D000DF92EF92FF920F931F93CF93DF9300D08C
:1019E00000D0CDB7DEB780E0882E82E0982E9CEE46
:1019F000A92E91E0B92E2EE1C22E22E0D22E38E29D
:101A0000E32E32E0F32E1AE01E0DD7018D917D01F9
:101A1000882331F1F401608171819E012F5F3F4F76
:101A2000AE014D5F5F4FD5018D919C910E94DB0609
:101A30008823B1F0D601EC91F0E0E75DFE4F208104
:101A4000213039F449816B818FE395E00E948B0C42
:101A500007C0022F49816B818FE395E00E94021E2F
:101A6000B2E08B0E911CE2E0AE0EB11CFFEFCF1A7C
:101A7000DF0A1E11CACF0F900F900F900F90DF91C9
:101A8000CF911F910F91FF90EF90DF90CF90BF907B
:101A9000AF909F908F9008952F923F924F925F92B8
:101AA0006F927F928F929F92AF92BF92CF92DF926E
:101AB000EF92FF920F931F93CF93DF93CDB7DEB7D3
:101AC0002F970FB6F894DEBF0FBECDBF1092090559
:101AD00010E002E0B6E0FB2E80E1E82E1A3091F033
:101AE0000E9433148823D1F300934705F0924805F0
:101AF000E092490566EF71E08FE395E00E94AD1931
:101B00001F5FECCF81E08093470588EE91E09093D2
:101B100076058093750588E4809377050E943314D9
:101B20008823E1F380910805813039F08091040524
:101B300081508E3FF8F483E04EC286E195E00E942A
:101B40007F1C2F960FB6F894DEBF0FBECDBFDF917E
:101B5000CF911F910F91FF90EF90DF90CF90BF90AA
:101B6000AF909F908F907F906F905F904F903F903D
:101B70002F9008958091020581508E3F08F42AC26B
:101B800090E08091050581508E3F08F028C282E0E8
:101B90008093980210919702212F48E952E06DE856
:101BA00072E08FE892E00E94970660918D0270913A
:101BB0008E0226E046E080918F02909190020E9472
:101BC0005D1F882351F0212F219548E952E06DE8EF
:101BD00072E08FE892E00E94970680918F029091C8
:101BE0009002879790938C0280938B0280918D0254
:101BF00090918E02459790938A02809389028091FA
:101C00008702882309F467C081508093870260911E
:101C1000960270E09B012F5F3F4F032E000C440B98
:101C2000550B719561957109072E000C880B990B66
:101C30000E94111400918B0210918C02012E000C55
:101C4000220B330BDC01CB01800F911FA21FB31FAE
:101C500090938C0280938B026091960270E09B01BE
:101C60002F5F3F4F032E000C440B550B7195619570
:101C70007109072E000C880B990B0E94111400911A
:101C8000890210918A02012E000C220B330BDC0119
:101C9000CB01800F911FA21FB31F90938A028093E4
:101CA00089022091F604269526951091F4048091DE
:101CB0009602289F90011124032E000C440B550B13
:101CC00060E070E0CB010E941114161B612F70E0E0
:101CD00085E00E94D81A6091890270918A028091F1
:101CE0008B0290918C020E94D11F60918D027091A5
:101CF0008E029E012B5F3F4FAE01495F5F4F809187
:101D00008F02909190020E94DB066D8161508F815D
:101D1000209198024EED51E081500E94DF20B12CBD
:101D2000A0E8AA2E8091DC02B81608F06DC00B2D39
:101D300010E09801220F331FF901E95CFD4F20806C
:101D4000318060908B0270908C02F901E95AFD4F4E
:101D5000408051808090890290908A0280918F0209
:101D600090919002A101481B590BCA0157FF03C073
:101D7000919581959109682FAC0155274034510503
:101D800014F06A2D681B6437E8F580918D029091FC
:101D90008E02B201681B790BCB0177FF03C09195CE
:101DA00081959109682FAC0155274033510514F0F6
:101DB00060E6681B603530F504521E4FF901E95AA0
:101DC000FD4F6F01A901495C5D4F7A0121E0A80137
:101DD000BF01C7010E9497068B2D0E946C058823C6
:101DE00009F409C12FEFA801B601C7010E949706A7
:101DF0000E94272B24E030E040E050E00E944B2B73
:101E0000D8016C93B3948ECF0E943B088091E90275
:101E1000882319F081508093E90280910605815052
:101E20008E3F08F0CFC08091070581508E3F08F4A7
:101E3000C9C02091E7023091E8022115310509F46B
:101E400061C18091E9028111BDC0E8E2F2E000E0E9
:101E500010E0302E819181114EC181E0F801E85DE2
:101E6000FD4F80838091EA02F801E25EFD4F80839E
:101E700090E0FC01E15EFE4F40814093E902215079
:101E800031093093E8022093E702FC01E65EFE4F41
:101E9000C080FC01E75DFE4F80814C2C80FD03C1BA
:101EA0004194A0908F02B09090020C2C000CDD08A1
:101EB000BFEFCB1ADB0A0D2C000CEE08FF08042C38
:101EC000000C550866087708A7019601C301B20106
:101ED0000E9411144801880C991CD401A451BE4FD2
:101EE000E3E0AE0EB11CE091EA02F0E0E75DFE4FE8
:101EF00020812695A21AB1086A0D7B1D6D937C93F3
:101F0000A0908D02B0908E02A7019601C301B2018C
:101F10000E9411142091EA02E22FF0E0A401405047
:101F20005E4F4A0153E0A50EB11CAF01475D5E4F05
:101F3000DA013C913695A31AB108A501460F571F47
:101F4000D4014D935C93D801AC5EBD4F8091980253
:101F50008C9330929102213009F0A7C080916205E4
:101F600080FFA6C08091EA02813009F4ADC0E09103
:101F7000EA02F0E0EB5EFE4F0081202F219548E958
:101F800052E06DE872E08FE892E00E94970610E060
:101F9000101771F060918D0270918E0226E046E07C
:101FA00080918F02909190020E945D1F811198C0D4
:101FB0008091EA02843031F481E08093960282E0DD
:101FC000809387028091070581508E3F08F0B8C04A
:101FD00082E0B7C081E08093980291E0D2CD8091F9
:101FE000030581508E3F20F0992309F4F6CDD2CD20
:101FF00010929802CFCD60E270E080E090E00E9405
:102000008219672B682B692B59F40E94272B24E037
:1020100030E040E050E00E944B2BF8016083F2CEAC
:1020200060E170E080E090E00E948219672B682BED
:10203000692B09F0E7CE62E070E080E090E00E945A
:102040008219672B682B692BB9F0C10180589F4F0B
:102050008619970960E870E00E9475292AE230E04D
:10206000281B390BC9011816190614F4E3E015C032
:1020700081E0D8018C93C6CEC201805A9F4F881947
:10208000990960E670E00E947529E8E1F0E0E81B3C
:10209000F90B1E161F0624F4E2E0D801EC93B2CE31
:1020A000D8011C92AFCE4094FCCE243009F456CF18
:1020B000EE0FFF1FED5EFE4F6591749140E086E1EB
:1020C00095E00E944B1C4ECF0E94272B60FF4FCF04
:1020D00040E06DE071E086E195E00E944B1C47CF47
:1020E00021E048E952E06DE872E08FE892E00E945A
:1020F00097061F5F4DCF0F5F1F4F0A30110509F084
:10210000A8CE60CFE091EA02E111E150E093EA024B
:10211000F0E0EE0FFF1FE25DFE4F80819181909312
:10212000E8028093E70284E18093E90280E091E095
:1021300090937605809375058AE28093770542CF68
:1021400081E08093970238E2432E32E0532E0CEE6A
:1021500011E040E0642E42E0742EE12CF12C58E0B6
:10216000C52EED86F2018081882309F49FC0F70116
:10217000E25EFD4FD0808D2D90E0FC01E75DFE4FCB
:102180002080FC01EC5DFE4F2081A7014C5E5D4F7D
:10219000B301C8010E949706D3016D917C91222D55
:1021A000422DF801808191810E945D1F811110C034
:1021B0009091DC0227E532E03A87298747E352E035
:1021C0005C874B8727E7822E22E0922E312C3BC082
:1021D000D2011C92B3E0DB1269C0F80180819181C9
:1021E0009093950280939402D3018D919C9190934A
:1021F000930280939202C092320240E06DE171E05E
:1022000086E195E00E944B1C51C0F40121914F01E1
:10221000A985BA85AD90BD90BA87A987EB85FC8565
:1022200041915191FC87EB87D3010D90BC91A02D7A
:10223000BF87AE87F801A081B181BD01620D731D1A
:10224000461757073CF0882DE7E7F2E08E1B891709
:10225000E0F22CC030E0420F531FA417B5079CF7E3
:102260004E855F85420D531DA416B50664F72A0DF1
:102270003B1D4E855F85421753072CF753E0D5125F
:1022800097C1B0939502A09394026E857F85709359
:10229000930260939202C092320240E06DE171E0DD
:1022A00086E195E00E944B1CD2011C92FFEFEF1AD1
:1022B000FF0A2FEF421A520A0E5F1F4F32E0630EE1
:1022C000711C4AE0E416F10409F04BCF0E94E30CC4
:1022D00080913202882309F48FC0815080933202AA
:1022E00084E08093960282E08093870266E070E04B
:1022F00080E090E00E9482191AE0160FC0909402CC
:10230000D090950268E070E080E090E00E94821931
:10231000A12EA694B12CDC01CB010497A109B1092F
:10232000B601680F791F7B01EA18FB0880909202C2
:102330009090930268E070E080E090E00E94821943
:10234000DC01CB010497A109B109B401680F791F21
:102350006B01CA18DB0800E0A12EB12C47018A0CE2
:102360009B1CAC0CBD1C8091DC02081738F5402F7B
:1023700050E0FA01E958FD4F208130E0440F551F2D
:10238000FA01E95AFD4F80819181FA01E95CFD4F24
:1023900040815181BA01620F731FE616F70664F49B
:1023A000481559054CF4280F391FC216D30624F4DA
:1023B0008A159B050CF400C10F5FD5CF9E012F5FDE
:1023C0003F4FAE014D5F5F4FB601C7010E94DB0674
:1023D000882391F082E080935F0580936005012F50
:1023E000212F49816B818FE395E00E94021E81E0DD
:1023F00080935F05809360050E94410C20918D02BF
:1024000030918E0260918F0270919002809135021E
:10241000909136024091330250913402FA0136967F
:102420006E177F071CF56A5F7F4F4E5F5F4F461741
:102430005707E4F4AC014A5F5F4F24173507B4F443
:102440002A5F3F4F02968217930784F480917805A4
:102450009091790505970CF0B5C08FE591E09093C8
:102460007605809375058AE2809377050E94860839
:10247000B6E5DB2E00E010E0EE24E394F090880255
:102480008F2D0F2C000C990B801791071CF024ED59
:1024900031E012C010925F051092600524ED31E02A
:1024A00040E06D2D8FE395E00E949D1CE0925F055A
:1024B000109260052AEC31E040E06D2D8FE395E04D
:1024C0000E949D1C0E5F1F4F57EFD50E62E3D61280
:1024D000D5CFF1100BC08091620580FD0EC082E067
:1024E0008093960281E08093870207C071E0F71223
:1024F00004C0F0929602F0928702F0FE10C0F7FC42
:10250000F394F594F09469E0F69E602D11246A5AD4
:1025100020EC31E040E08FE395E00E949D1C80912B
:10252000E7029091E802892B11F00E94011F0E949E
:10253000722410E002E0F4E0FF2EA3E0EA2E809186
:10254000DC02181708F0EACA80918D0290918E0281
:1025500060918F0270919002212F30E0F901E958CB
:10256000FD4FB0804B2D50E0220F331FF901E95A87
:10257000FD4F0190F081E02D295C3D4FD9012D9157
:102580003C916901C40ED51E6C157D057CF46A5F13
:102590007F4F2617370754F44E0F5F1F8417950798
:1025A0002CF40696E817F9070CF455C01F5FC7CF47
:1025B0006D850E941B0778CE60919102802F0E944A
:1025C0001B07FACE8091EA02843088F484E591E01A
:1025D00090937605809375058AE28093770540E0B5
:1025E00062E371E086E195E00E944B1C09C087E23E
:1025F00091E090937605809375058AE28093770544
:10260000809178059091790505979093790580934D
:1026100078050E94AD08E091EA028E2F90E00497C1
:1026200014F4EF5F01C0E4E0E093EA02F0E0EE0FA3
:10263000FF1FE25DFE4F808191819093E8028093BD
:10264000E70280918802853014F48F5F01C086E034
:10265000809388020BCF809188029FEF980F909310
:10266000880200939602F092870266E0B61205C0D7
:10267000825080938802E092960240E06AEB71E01B
:1026800086E195E00E944B1C812F0E94FF058091FE
:10269000880287FF8BCF10E084E5D82EFF24F394C7
:1026A0009CE0E92E0E9433148823E1F30E943B084A
:1026B0000E94E30C0E94410C0E9486088091E70270
:1026C0009091E802892B11F00E94011F0E94722450
:1026D0006091890270918A0280918B0290918C02A4
:1026E0000E94D11F6D8161508F81209198024EED23
:1026F00051E081500E94DF2010925F05109260052A
:1027000000E3212F40E060E08FE395E00E94021E8D
:102710006D2D611B212F40E08FE395E00E94021E8A
:10272000F0925F0510926005E0924805F09249052D
:102730006FEA71E08FE395E00E94AD191E5F1E33D2
:1027400009F0B0CF1CE0FF24F39408E20E94331498
:102750008823E1F320917805309179058091A102D9
:102760009091A20282179307A4F462E070E080E0E7
:1027700090E00E9482196E5F6093480562E070E00D
:1027800080E090E00E9482196093490561EA71E05F
:1027900006C010934805F092490566E971E08FE3A1
:1027A00095E00E94AD1910924805109349056BE819
:1027B00071E08FE395E00E94AD196091780570910A
:1027C00079058FE395E00E94FF236EE771E08FE3C8
:1027D00095E00E94AD196091DA027091DB028FE3FF
:1027E00095E00E94FF2366E771E08FE395E00E9489
:1027F000AD1910924805009349056DE671E08FE32D
:1028000095E00E94AD1980910605813009F09ECFB8
:1028100086E195E00E94841C0E94FA087FC90E940C
:10282000CD2ACF92DF92EF92FF920F931F93621700
:1028300073078407950784F489019A016B017C0171
:10284000C901B8016C197D098E099F090E9482197E
:102850006C0D7D1D8E1D9F1D1F910F91FF90EF90A0
:10286000DF90CF9008954F925F926F927F928F92F8
:102870009F92AF92BF92CF92DF92EF92FF920F930F
:102880001F93CF93DF9300D000D01F92CDB7DEB758
:1028900040917105509172056091730570917405B6
:1028A0002FB7F8948091E3029091E402A091E502A1
:1028B000B091E6022FBF481B590B6A0B7B0B80912E
:1028C000700590E0A0E0B0E000916C0510916D05FE
:1028D00020916E0530916F0584179507A607B707FD
:1028E00030F4011511052105310509F0F4C2012B61
:1028F000022B032B09F0EDC28091080581508E3F19
:1029000008F580910705813011F580911B058F5FD7
:1029100060911C0587FD09C0082E000C990B70E022
:102920006F5F7F4F0E947529682F60931B0581EAB6
:1029300098E0909376058093750588E480937705F9
:102940000E94E8218091080581508E3F70F48091AB
:102950000605813009F06BC384E998E09093760511
:102960008093750588E48093770580E00E94DB22E0
:1029700080911705882309F4ADC080912B05811142
:10298000A9C08091230590912405E0912805F0913C
:102990002905EE0FFF1FE80FF91F459154914115CE
:1029A000510501F520912705222331F010922905C8
:1029B00010922805FC0114C010921705809116058D
:1029C000882341F080E00E94DB22E0912805F0910D
:1029D00029052FC060E086E195E00E943A1C7AC08C
:1029E000459154919A01369527953695279540FF44
:1029F00051C0CA01B6E096958795BA95E1F78F71F7
:102A0000952F96959695969590512F70223071F14D
:102A1000F8F4211117C08B3008F08AE080932C0560
:102A2000E0912805F09129053196F0932905E0936E
:102A30002805EE0FFF1F8091230590912405E80FD4
:102A4000F91FCECF213061F760E00E941C23E8CF50
:102A50002330B1F0243021F720911A05829F802D78
:102A600011248093330590933405DACF20911A0511
:102A7000829F802D112480932F0590933005D0CF15
:102A800020911A05829F802D112480933105909307
:102A90003205C6CF2F7320932A0580911A05859F92
:102AA000802D112480932B0510923B0510923A053E
:102AB0001092390581E080932D058093DE021092FB
:102AC0002E0580912805909129050196909329055E
:102AD0008093280580912D05882309F4F3C0809107
:102AE0002B05811106C060E086E195E00E943A1C4A
:102AF000E9C0815080932B0580913B05811148C02E
:102B00002091390530913A052F5F3F4FC901880F59
:102B1000991FE0913505F0913605E80FF91F659191
:102B20007491862F877080933C05AB0163E05695C6
:102B300047956A95E1F7CA0196958795972F9695DF
:102B4000969590933D058F7390911A05899F802DDE
:102B5000112480933B0541704093E20230933A0583
:102B6000209339058091370590E02817390780F0C8
:102B700020913805222339F0821B910990933A0560
:102B80008093390505C060E086E195E00E943A1C1B
:102B900080913B05815080933B0580912E0521E07B
:102BA000280F20932E0540912A0530913D05340FC2
:102BB00080912205380F3093180560913105662306
:102BC00071F070E0822F022E000C990B0E94752983
:102BD00080913205869F300D112430931805809125
:102BE000180590E0849664E270E00E947529809355
:102BF000180530912C053093190560912F05662337
:102C000081F0062E000C770B822F022E000C990B00
:102C10000E94752980913005869F300D11243093D4
:102C20001905609133056623A1F0822F220F990BBD
:102C300070E00E947529CB0162E070E00E94752966
:102C40002091340590911905289F900D112490939F
:102C50001905809119054F3341F08A300CF089E055
:102C600087FD80E08093190502C010921905F89441
:102C7000E0911805F0E0E054F94FE491E093E102AF
:102C80003091190520913E053203900111244091A5
:102C90003C054203C001439F900D112400901B0589
:102CA00002C0880F991F0A94E2F797FF02C081586B
:102CB0009F4F880F892F881F990B8093E002809384
:102CC000DF02789480917705882309F456C08C3010
:102CD00020F49CE0E92EE81A01C0E12CFF24F394D3
:102CE000F092470510925F051092600530914405FF
:102CF0001DE2D12ED31ADE0C03E0030F2EE44D2D7E
:102D000063E08FE395E03D830E94021E3D810CEF5E
:102D1000030F33E0D30E202F41E06D2D80E50E949C
:102D2000A423202F42E06D2D83E00E94A423F09283
:102D30005F05F09260058091440523E0280F612F24
:102D4000681B6E0D44E580E00E94572384E0809369
:102D5000480580914405E81A8E2D815D80934905D0
:102D600060917505709176058FE395E00E94AD192D
:102D70008091770581508093770580910D05909122
:102D80000E05892B09F47DC011E010935F051092A8
:102D900060059091430585E5891B80934805109255
:102DA000490560910A05613009F44CC030F080910A
:102DB0000905653008F05EC059C060E086E195E025
:102DC0000E943A1C109217051093470562E177E0C4
:102DD0008FE395E00E94891C10920E0510920D055C
:102DE0001092450518EA0E9433148823E1F364E049
:102DF00077E08FE395E00E94AD1940910B0550916B
:102E00000C0560E070E02AE08FE395E00E94E6198F
:102E10006FEE76E08FE395E00E94AD19612F629529
:102E20006F7070E08FE395E00E94FF2364EE76E020
:102E30008FE395E00E94AD1980910605813009F07D
:102E4000FCC01FC08091620590916305A09164054C
:102E5000B09165058F709927AA27BB270897A10510
:102E6000B10510F467E009C068E707C0882349F09E
:102E70006B5F03C0882329F06FE28FE395E00E9427
:102E8000A6190E9462228091450581110EC088EF2B
:102E900091E0E1EFF2E0DF019C011D922150304012
:102EA000E1F710924805109249050E944E1B60936D
:102EB0006C0570936D0580936E0590936F0520915E
:102EC000680530916905621B730B70936705609309
:102ED000660580E0CCC02FB7F8948091E302909112
:102EE000E402A091E502B091E6022FBF20917005A7
:102EF000820F911DA11DB11D8093710590937205E4
:102F0000A0937305B0937405809162059091630559
:102F1000A0916405B09165050196A11DB11D809336
:102F2000620590936305A0936405B09365051092C4
:102F30006C0510926D0510926E0510926F050E943F
:102F40004E1B609368057093690580936A059093A2
:102F50006B058091F2049091F3042FE0289F80018B
:102F6000299F100D112485E10E94371B800F911FAE
:102F700024E0969587952A95E1F79093F304809342
:102F8000F2042091F104222309F44BC06091F5046E
:102F9000262F30E040E050E029833A834B835C8366
:102FA000C090F604D12CE12CF12C4091F904509101
:102FB000FA044A01A12CB12C2091F7043091F804B5
:102FC0002901612C712C8217930728F09C01481766
:102FD000590708F49A01C901A0E0B0E09C01AD01D5
:102FE000241935094609570969817A818B819C81A9
:102FF0006C197D098E099F090E945929A501940128
:1030000024193509460957090E944B2BC20ED31EBD
:10301000E41EF51EC092F4046C2D70E085E00E9461
:10302000D81A0E94EF210E94352481E020C0893205
:1030300009F09BCC0E94A22298CC115009F0D3CE6B
:1030400060E070E085E00E94D81A83B7817F8460D9
:1030500083BF83B7816083BF83B7816083BF889557
:1030600083B78E7F83BF83B78E7F83BFBCCE0F9025
:103070000F900F900F900F90DF91CF911F910F91B4
:10308000FF90EF90DF90CF90BF90AF909F908F9088
:103090007F906F905F904F900895CF92DF92EF9264
:1030A000FF920F931F93CF93DF9380916105882345
:1030B00009F4D0C081E08093470510924605109234
:1030C00045051092090580935F0580936005CFEB5D
:1030D000D6E01CE00E9433148823E1F3FE018491C2
:1030E000882319F00091440501C000E02DE235E08D
:1030F00040E060E08FE395E00E949D1C4CE0400FB3
:103100002DE935E060E08FE395E00E949D1C109270
:103110004805109349056FEB76E08FE395E00E9438
:10312000AD1980914305982F990F890F81958D5A7C
:103130008093480580914405982F990F890F8195B8
:10314000835D809349058091620584FF03C069E235
:1031500075E002C065E275E08FE395E00E942F1AEA
:1031600080914305982F990F890F81958D5A8093EF
:103170004805809149058F5F8093490580911B0523
:10318000882319F061E275E002C06DE175E08FE31C
:1031900095E00E942F1A80914305982F990F890F6F
:1031A00081958D5A80934805809149058F5F809362
:1031B000490569E175E08FE395E00E942F1A80913F
:1031C00007058130A1F480911B058F5F60911C057C
:1031D00087FD09C0082E000C990B70E06F5F7F4FD0
:1031E0000E947529682F60931B050E94E821809139
:1031F00006058130A9F080916105482F50E060E01C
:1032000070E0C0906205D0906305E0906405F09096
:103210006505C416D506E606F706A0F08F3F91F0C7
:103220008FEF8093610560E086E195E00E943A1C93
:103230001092170586E195E00E94841C81E080933E
:10324000090508C080910805813009F043CF0E942C
:10325000A22240CFDF91CF911F910F91FF90EF906D
:10326000DF90CF900895CF92DF92EF92FF920F936D
:103270001F93CF93DF936C017A018B01C0E0D0E004
:10328000CE15DF0589F0D8016D918D01D601ED9144
:10329000FC910190F081E02DC6010995892B11F474
:1032A0007E0102C02196ECCFC701DF91CF911F9123
:1032B0000F91FF90EF90DF90CF900895282F862FE9
:1032C0006CE00E946929E22FEF70F0E083E0F59551
:1032D000E7958A95E1F7E90FF11DE90FF11DE1543A
:1032E000F74FE491F0E0277080E890E002C09595F8
:1032F00087952A95E2F7E823F92381E0EF2B09F47B
:1033000080E00895CF93DF9300D000D0CDB7DEB733
:10331000611571058105910579F09B01AC01698307
:103320003A834B835C830E94272B29813A814B810E
:103330005C810E944B2B03C060E070E0CB010F90DA
:103340000F900F900F90DF91CF910895DC01ED91D8
:10335000FC910190F081E02D0994EF92FF920F9380
:103360001F93CF93DF938C017B01C0E0D0E0F70186
:10337000EC0FFD1F6491662361F0D801ED91FC9183
:103380000190F081E02DC8010995892B11F021965B
:10339000EECFCE01DF91CF911F910F91FF90EF9073
:1033A00008956115710579F0FB0101900020E9F79E
:1033B0003197AF01461B570BDC01ED91FC91028068
:1033C000F381E02D099480E090E008954F925F92A0
:1033D0006F927F92EF92FF920F931F93CF93DF93A1
:1033E000CDB7DEB7A1970FB6F894DEBF0FBECDBF45
:1033F0007C01FA01CB0119A2223008F42AE08E01E7
:103400000F5D1F4F422E512C612C712CBF01A30167
:1034100092010E947D2BF901CA01015011096A3005
:1034200014F4605D01C0695CD8016C93232B242BDC
:10343000252B61F7B801C7010E94D119A1960FB6DB
:10344000F894DEBF0FBECDBFDF91CF911F910F91DA
:10345000FF90EF907F906F905F904F9008950F9343
:103460001F93CF93DF93EC010E94AD198C0160E4B0
:1034700071E0CE010E94D119800F911FDF91CF9191
:103480001F910F910895833081F028F4813099F0D5
:103490008230A1F008958730A9F08830B9F08430E7
:1034A000D1F4809180008F7D03C0809180008F7760
:1034B00080938000089584B58F7702C084B58F7D96
:1034C00084BD08958091B0008F7703C08091B000D3
:1034D0008F7D8093B00008951F93CF93DF93282FA3
:1034E00030E0F901E258F64F8491F901E659F64FC0
:1034F000D491F901EA5AF64FC491CC23C9F0162FA2
:1035000081110E94431AEC2FF0E0EE0FFF1FEB5BDE
:10351000FD4FA591B4918FB7F894111105C09C91FE
:10352000ED2FE095E92302C0EC91ED2BEC938FBFDA
:10353000DF91CF911F910895CF93DF9390E0FC012D
:10354000E659F64F2491FC01EA5AF64F84918823FC
:1035500061F190E0880F991FFC01E55CFD4FC5917A
:10356000D491FC01EB5BFD4FA591B491611109C0B1
:103570009FB7F8948881209582238883EC912E232D
:103580000BC0623061F49FB7F8943881822F809528
:1035900083238883EC912E2B2C939FBF06C08FB77B
:1035A000F894E8812E2B28838FBFDF91CF91089567
:1035B0001F93CF93DF93182FEB0161E00E949C1AB9
:1035C000209711F460E004C0CF3FD10539F461E0E9
:1035D000812FDF91CF911F910C946C1AE12FF0E0B5
:1035E000E258F64FE491E330F9F048F4E130B9F0F5
:1035F000E230A1F584B5806284BDC8BD34C0E73037
:10360000E9F0E83019F1E43049F5809180008062FA
:1036100080938000D0938B00C0938A0024C084B52F
:10362000806884BDC7BD1FC0809180008068809382
:103630008000D0938900C093880015C08091B000AD
:1036400080688093B000C093B3000DC08091B0003B
:1036500080628093B000C093B40005C0C038D1052B
:103660000CF0B5CFAFCFDF91CF911F9108958E3081
:1036700008F08E508770806480937C0080917A007F
:10368000806480937A0080917A0086FDFCCF8091DF
:1036900078002091790090E0922B08953FB7F8943C
:1036A0008091ED029091EE02A091EF02B091F002B4
:1036B00026B5A89B05C02F3F19F00196A11DB11D8D
:1036C0003FBFBA2FA92F982F8827820F911DA11DC8
:1036D000B11DBC01CD0142E0660F771F881F991F05
:1036E0004A95D1F708958F929F92AF92BF92CF9251
:1036F000DF92EF92FF926B017C010E944E1B4B0107
:103700005C01C114D104E104F104F1F00E944E1BEC
:10371000DC01CB0188199909AA09BB09883E9340AD
:10372000A105B10570F321E0C21AD108E108F10842
:1037300088EE880E83E0981EA11CB11CC114D10430
:10374000E104F10419F7DDCFFF90EF90DF90CF9007
:10375000BF90AF909F908F9008951F920F920FB6D9
:103760000F9211242F933F938F939F93AF93BF9307
:103770008091E3029091E402A091E502B091E6020B
:103780003091EC0223E0230F2D3720F40196A11D88
:10379000B11D05C026E8230F0296A11DB11D20937F
:1037A000EC028093E3029093E402A093E502B093CD
:1037B000E6028091ED029091EE02A091EF02B091AD
:1037C000F0020196A11DB11D8093ED029093EE02CF
:1037D000A093EF02B093F002BF91AF919F918F91B0
:1037E0003F912F910F900FBE0F901F9018951F9231
:1037F0000F920FB60F9211242F936F937F938F9395
:103800009F936091E002662359F18091EB028F5FF4
:103810008093EB029091E102891710F12091DE0272
:1038200081E028272093DE021092EB028091E202D1
:10383000882369F08091000193E4899F802D1124F1
:10384000895B809300010E9469299093DF02222303
:1038500029F08091DF028093B40002C080E0FBCFAA
:103860009F918F917F916F912F910F900FBE0F902D
:103870001F901895FC0161110DC0178A158A14A2BA
:1038800013A2108E1092DF021092E0021092DE025C
:103890001092B4000895EF92FF920F931F93CF936D
:1038A000DF931F92CDB7DEB77C018B01411105C0BC
:1038B00060E049830E943A1C498150E0FA01EE0F12
:1038C000FF1FEE0DFF1D16870587DA011996AA0F57
:1038D000BB1FAE0DBF1D1D921C92F701E40FF51F1B
:1038E00081E0818389E0868B118E138E158E0F9077
:1038F000DF91CF911F910F91FF90EF90089540E0DD
:1039000067EF78E00C944B1C40E06FEE78E00C948D
:103910004B1CDC01FB0184918F5F14968C931497F0
:103920003196E491EF5F1596EC9315976E5F7F4F9C
:103930005F967C936E935E9708954F925F926F921D
:103940007F928F929F92AF92BF92CF92DF92EF922F
:10395000FF920F931F93CF93DF93F901C490319699
:103960005491EC0108A164350CF018C10C2C000C2A
:10397000DD08A62F062E000CBB0B7D01EC0CFD1CF8
:103980001E141F040CF00AC140330CF007C1A52E11
:10399000842E042E000C9908F401E50FF11D57FD4B
:1039A000FA951E161F060CF0F9C02E5F3F4FE60178
:1039B0002796D7FD279673E0D595C7957A95E1F7B9
:1039C00047FF0AC0A52EA40EC89DA001C99D500D99
:1039D0001124241B350B40E0EA2D0A2C000CFF0BB0
:1039E000E40FF11D47FDFA95F1971CF050E3A52E69
:1039F000A41A67FD60E0F701E535F10514F0E4E590
:103A0000F0E07E2FFC01D484D426862F062E000CF5
:103A1000990BFC01EA1BFB0BDF017F01F7E0EF22B2
:103A2000FF24E0E8F0E002C0F595E795EA94E2F7BC
:103A30001E2FB7FD179653E0B595A7955A95E1F758
:103A40002A0F3B1FE42FE77051E001C0550FEA95A4
:103A5000EAF7459545954595B4E54B02800D911DD6
:103A600011248F509D4FC12C0A2C000CBB089924A7
:103A700093942E015524EC2DF0E0EA15FB050CF093
:103A80008DC0F90144910130E1F47C01A12F862E13
:103A9000881AB82DBE0DB71708F077C0B42FBA2317
:103AA00021F0E701B881B52BB883B0E0B595A795B3
:103AB000109719F431964491A0E8DFEFED1AFD0A52
:103AC000E8CF01111FC0752E70947C01A12FF90160
:103AD000862E881AB82DBE0DB71708F056C0B42F21
:103AE000BA2321F0E701B881B721B883B0E0B595DA
:103AF000A795109719F431964491A0E8DFEFED1ADD
:103B0000FD0AE8CF033031F07C01A12FF901862EA8
:103B1000881A37C0752E7094862E7C01A12FF9016A
:103B20008716D8F4B42FBA2359F0E701B881682C6E
:103B30006D2460FE02C0B52B02C0B721E701B88337
:103B4000B0E0B595A795109719F431964491A0E887
:103B50008394DFEFED1AFD0AE3CFD92416C0B42F0A
:103B6000BA2321F0E701B881B527B883B0E0B59555
:103B7000A795109719F431964491A0E8DFEFED1A5C
:103B8000FD0AB82DBE0DB71750F3550F19F48C5A16
:103B90009F4F51E0C394240D351D6DCFDF91CF9120
:103BA0001F910F91FF90EF90DF90CF90BF90AF905B
:103BB0009F908F907F906F905F904F900895DF92CD
:103BC000EF92FF920F931F93CF93DF931F92CDB786
:103BD000DEB78C01D62EF42EE12CE21654F46E2DB5
:103BE0006D0D4F2DC80129830E948B0CE394298110
:103BF000F4CF0F90DF91CF911F910F91FF90EF9035
:103C0000DF900895DF92EF92FF920F931F93CF936F
:103C1000DF937C01D62FD22EC42F002E000C110B67
:103C2000040F111D47FD1A954C2F0C2E000C550B3F
:103C30004017510744F42D2D4C2F6D2FC7010E94C2
:103C4000DF1DCF5FF1CFDF91CF911F910F91FF90DB
:103C5000EF90DF9008956F927F928F929F92AF9234
:103C6000BF92CF92DF92EF92FF920F931F93CF9369
:103C7000DF93EC0188A064350CF080C040330CF079
:103C80007DC0EC81F0E031970E9FC0010F9F900D39
:103C90001124860F911D67FD9A95181619060CF0D0
:103CA0006DC0ED81E09FF0011124E40FF11D47FD8F
:103CB000FA951E161F060CF061C0102FE42EF62E8A
:103CC000962EB62EC22ED12CEB2DEF190E2E000CF7
:103CD000FF0B8C8190E0E817F9070CF04EC00197BC
:103CE000E817F90779F0C89E9001C99E300DD89E5B
:103CF000300D1124E20FF31F8E8D9F8DE80FF91FF9
:103D0000749001C0712C6E2CAE2C2A2D2E19022E0F
:103D1000000C330B8D8190E0281739075CF570FE9D
:103D200010C0113031F44A2D6B2DCE010E948B0C46
:103D30001DC0012F212F462D692DCE010E94021E8C
:103D400015C089A198A1891789F088A3113031F491
:103D50004A2D6B2DCE010E948B0C07C0012F212F05
:103D6000462D692DCE010E94021E88A27694A3944E
:103D7000610ECBCFB394910EA7CF88A2DF91CF91E4
:103D80001F910F91FF90EF90DF90CF90BF90AF9079
:103D90009F908F907F906F9008950F93CF93DF93B4
:103DA000EC016A3019F42D8198851FC06D3019F12E
:103DB000262F08854A8569850E942B1E28853C810F
:103DC0008985329F800D112489879F81992399F0DD
:103DD000082E000C990B44E550E0239F401951092F
:103DE0001124481759073CF49D818A85299F800D2D
:103DF00011248A87198681E090E0DF91CF910F919D
:103E000008950F93109248059091440580E3891B13
:103E100080934905E091EA02F0E0EE0FFF1FEB51BD
:103E2000F74F659174918FE395E00E94AD19209151
:103E3000E902233038F002E04EE26EEF8FE395E0C6
:103E40000E94021E9091EA02209144058091430550
:103E5000992309F14091E7025091E8024436510557
:103E600030F4982F4A30510518F4990F01C090E0B2
:103E7000382F330F830F981B9C5A9093480580E38B
